:030000000219FDE5
:03000B000200AA46
:03002B000201606F
:03005B000202F6A8
:030073000202DCAA
:1000800002030406080C10182030406080040608A3
:100090000C10182030406080A0C000070F1F3F0DDB
:1000A0000D0403060D0502030202C2AFC0D0C0E07A
:1000B000206217E5256002E473E525F4F58A758B67
:1000C00000D262D0E0D0D0D2AF3285268AC262E5BB
:1000D00026F46030758B00D0E0D0D0C295C294C2B7
:1000E00093D2AF32C295C294C293206E0D20660A9D
:1000F0007405D5E0FDE57EF45290758B00D0E0D01C
:10010000D0D2AF32758A00C28DD26201FA01B93005
:100110006805206602D29501B9306805206602D2D2
:100120009401B9306805206602D29301B9D29230A9
:10013000680A2066077403D5E0FDD29501B9D29113
:1001400030680A2066077403D5E0FDD29401B9D265
:100150009030680A2066077403D5E0FDD29301B998
:10016000C2AFC2AD53E6EFC0D0C0E0D2D3D2AFC26F
:10017000CEE52A6007207449152A21C1780079004C
:1001800020742EE580307E01F430E70278FF53DAE8
:10019000CF207E0343DA20307E0343DA10C2D8C278
:1001A00071E580307E01F430E70279FFC3E8997091
:1001B000CB306103752A40207403752A40885FD2D2
:1001C0007020740DE52B6004152B21D143DA01C298
:1001D000D820700221E4A85F206102C2702074025E
:1001E00021E288227882B60403852224C3E525947F
:1001F000404002D26420CF0AD0E0D0D043E610D2F3
:10020000AD32C2CF053A7802E52A60053074021596
:100210002AC3E55F94014005756200412E756300B5
:10022000756C00E5622401F56250037562FF798206
:10023000B7020D306D1DC3E52294324016854D2264
:100240007982B7030E306D0BC3E5229432400479F6
:100250008E8722C3E523952260084004152341625E
:100260000523D8CA056CE56C7002156CD56D6375F5
:100270006D017805C3E56C956E4057C3E56C956FCD
:1002800050087801756D03020296C3E56C957050B5
:10029000057801756D01C3E5659524401E7982B727
:1002A000040241C7206D14852465E56C0460038554
:1002B0006E6C756D0175233C0202D2E56528500510
:1002C0007565FF41C7F565E5650470067563FF75E3
:1002D0006CFFD0E0D0D043E610D2AD32C2AFC0D078
:1002E00053E67FC260759100855694855795759148
:1002F00004D0D0D2AF32C2AF53E6EFC2ADC0D0C04F
:10030000E0C0F0D2D3D2AFA8FBA9FCC2D8307102B2
:10031000615D53DACF207E0343DA10307E0343DA87
:1003200020D271E580307E01F420E7026134882715
:100330008928A14253DACF207E0343DA20307E039E
:1003400043DA10C2D8C271307402A12E7800E58061
:10035000307E01F430E702A12E885FA11653DACF78
:10036000207E0343DA20307E0343DA10C27120611D
:1003700002813653DACF207E0343DA10307E034306
:10038000DA20C2D8D271885A895BC3E89558F8E957
:100390009559F97B007E087A00C3E8948CE99400B3
:1003A0005005755E008128882178A2E6A821605555
:1003B000C3E894C8E994005008E4D2E4FB7A0A81C7
:1003C00003C3E89468E994015008E4D2E3FB7A0F90
:1003D0008103C3E894D0E994025008E4D2E2FB7AA6
:1003E0001E8103C3E894A0E994055008E4D2E1FB20
:1003F0007A3C8103C3E89498E994085008E4D2E079
:10040000FB7A787E00C3E8955CFCE9955DFD30E7FA
:100410000AECF42401FCEDF43400FD755E00C3EC3D
:100420009AED9E5003755E01885C895D855A5885FA
:100430005B597802A116C3E89527F8E99528F930A9
:100440007C0281FA307B0281FA307A0281F32075D6
:10045000028159E9FDE8FC8178E9C313F9E813F852
:1004600030790281F3E9C313F9E813F83078028197
:0F047000F3E9C313FDE813FC20612CC3EC941CCB
:10047F00ED94024002818FED701EC3EC94C85018AA
:10048F000529E52970021529C3E529940A5002A10F
:10049F002E755F00D270A12EE52960021529740018
:1004AF00207F037896E624FAFEE43400FFC3EC9E27
:1004BF00FCED9FFD50067800790081FAC3EC94FFA4
:1004CF00ED9400400678FF790081FAEC8575F0A471
:1004DF00C5F0A2F733F87900400302051678FF79CB
:1004EF0000020516E9C313F9E813F8307C0EE96032
:1004FF000278FFC3E81338F8E43400F9C3E894FF37
:10050F00E99400400278FF885FD270206102A12E2B
:10051F00741FF4552F4BF52FC274EB7002D2747504
:10052F002A40307403752A0A306102A142207403F5
:10053F0053DAFE207403752B20D0F0D0E0D0D0D248
:10054F00AD43E61032790102057279030205727923
:10055F000A020572791E020572796402057279C862
:10056F000205727817E4D5E0FDD8FAD9F6227A148D
:10057F007B780205997A107B8C0205997A0D7BB4F2
:10058F000205997A0B7BC80205997902B27DE4D2F4
:10059F0091D5E0FDD294D5E0FDC294D5E0FDC29196
:1005AF00D5E0FDD295E576D5E0FDC2957496D5E000
:1005BF00FDD9D9EAF8D5E0FDD8FBDBCED29122C325
:1005CF007C007D0075F00005F0EA33FAEB33FB5049
:1005DF00F6EB13FBEA13FAC3E9FFE8FEE89AF8E932
:1005EF009BF95004EFF9EEF8B3EC33FCED33FDD586
:1005FF00F0DFEDF9ECF822E889F08A20D2D4F8A9DF
:10060F00F07B0030F70B7BFFF42401F8E9F43400A2
:10061F00F9E88520F0A4ADF0F8E98520F0A4AFF05B
:10062F00FEED2EF974003FFA7C04C3EA13FAE913C6
:10063F00F9E813F8DCF48BF030F70AE8F42401F84A
:10064F00E9F43400F9E889F0C2D4F8A9F0227882ED
:10065F00B604030206FCC3E55F9419401EE52D5452
:10066F00067018206D3678057994E7146007780ABC
:10067F001460027812C3E54198401F306D098567F9
:10068F0065756CFF756D01852224E4F545F546F51A
:10069F0047F548F549C26D0206FCD26D7994E7140F
:1006AF007013E523F43333F913F8E9540104F9E82F
:1006BF0054FE0206F0E714147014E523F4333333B9
:1006CF00F913F8E9540304F9E854FC0206F8E5239A
:1006DF00F433333333F913F8E954070404F9E854C6
:1006EF00F8C39440F8E99400F98845894622C3E598
:1006FF004113F9E54013F8C3E54598F8E54699F934
:10070F00500CC3E89480E994FF4016020734C3E805
:10071F00947FE994005003020734787F7900020731
:10072F0034788079FF884A894B22E54A2547F8E5D6
:10073F004B3548F9854B20E4300701F43549FA3041
:10074F00E709C3EA94F04015020772C3EA940F5009
:10075F000302077278FF79FF7A0F02077278007928
:10076F00007AF0C3E5249564500AC37401952450B0
:10077F000B020790E54B20E70E020790E54B30E7A1
:10078F0006884789488A492278A4E6FAC3E54A339E
:10079F00F8E54B33F9D106E930E70BC3E89480E96C
:1007AF0094FF4013E1CAC3E8947FE994005002E13B
:1007BF00CA787F7900E1CA788079FFE820E715C30E
:1007CF00E52398F84009C3E8940140030207F17844
:1007DF00010207F1E8F424012523F840030207F191
:1007EF0078FF884C2278A5E6FAA848A949D106E9EE
:1007FF0030E70CC3E89401E994FF4016020825C3C3
:10080F00E894FFE99400500302082578FF7900026D
:10081F000825780179FFE920E715C3E54C98F840E2
:10082F0009C3E89401400302084C780102084CE820
:10083F00F42401254CF8400302084C78FF88242249
:10084F0078FFC26420693D206A12D264C3E54194E7
:10085F000A4009C3E52594405002C26479A1E760BC
:0E086F0023E541601F74FF8541F0848539F058
:10087D00306A0375F005A4F8C5F0600278FFC3E88F
:10088D0095675002A867886622C3E5409440E5410C
:10089D009401E56650031401A7046002F566227801
:1008AD0083E6F520120F4575E89012055475E89012
:1008BD00E5E820ECFBA8BDA9BE120FDF75715575DB
:1008CD007200C3740013FD7455606613FC74552CCF
:1008DD00FC74003DFDECFAEDFBC3E89AE99B401476
:1008ED00E5712455F571E5723400F572EA2CFAEBD9
:1008FD003DFB80E5AE71AF72C3E57213F9E571137F
:10090D00F8C3E913F9E813F87A03C3E913F9E81307
:10091D00F8DAF7AA201A70097571007572000209CC
:10092D003E1AEA6008EE28FEEF39FFDAF88E718F75
:10093D00722275E890227883E6FFE5E820ECF7A8AF
:10094D00BDA9BE0573C3E57394084052757300E9E4
:10095D00FA79A0E76044EA7007E574601B02097933
:10096D00C3E895746010E5745006600C1402098597
:10097D000460F9020985E574F574C3946D401B7527
:10098D0064C0C394044013756480C39404400B7514
:10099D006440C39404400375640075BB0622EFC325
:1009AD009401601F7455601BC3E894FFE9940350D4
:1009BD0012C3E89571E995725009E564600C1564F0
:1009CD000209D7E564F460020564A864C3E52498C0
:1009DD005002A824C3E89565400AA865E565F46052
:1009ED000385656488258826E573B4070375BB10F8
:1009FD0022743279A687F0A4C5F0A2F733F8C3E8C4
:100A0D0095644002A86488228824882588268867F2
:100A1D00227540007541F022C2AF75C820A8CCA93F
:100A2D00CDAA3A30CF010A75C824D2AFAB3BAC3C4E
:100A3D00883B893CC3E89BF8E99C206908F930673D
:100A4D0002613A4197AD3D8A3DF9EA9DFA6004781D
:100A5D00FF79FFAE3EAF3F8B3E8C3FC3EC9FFCC397
:100A6D00E99CF542A83BA93CC3E89EF8E99FF9C370
:100A7D00E54113FBE54013FAE82AF540E93BF54162
:100A8D0050067540FF7541FF41E1AA40AB41AC40B6
:100A9D00AD417E047F02C3EB940440021E1FC3EBE5
:100AAD00940840021E1FC3ED13FDEC13FCDEF7C3CB
:100ABD00EA9CFAEB9DFBEF6009C3E913F9E813F823
:100ACD00DFF7EA28FAEB39FB8A408B4150067BFFB2
:100ADD008B408B41C3EB94025002D2673069047F87
:100AED0003610C7892E6FFC3E537948240110FC382
:100AFD00E53794A040010FC3EF940640027F057EB9
:100B0D0004E541C4540FF9E541C454F0F8E540C47F
:100B1D00540F28F8C3E89EFAE99400FB4009C3EA94
:100B2D009402EB940050047A02E4FB6186AA40AB78
:100B3D0041EBC4FEEAC4540F4EFCC3EA9CFAEB949D
:100B4D0000FBC3E813C313F8EA28FAEB3400FB8A61
:100B5D00408B41C3EB94024002C2677804EBC4FEA4
:100B6D007B00EAC4540F4EFAC3EA98FA4005C394C9
:100B7D000250027A027892E6FF3060026186855259
:100B8D0056855357D26043E680C3E49AF8E49BF947
:100B9D003067028120E8FAE9FBD3E913FDE813FC85
:100BAD0088528953C3EF94036038EF20E00DE82C91
:100BBD00F8E93DF9ECFAEDFB020BDBE828F8E93931
:100BCD00F9C3E82402F8E93400F97AFE7BFFC3EF9C
:100BDD009403400E8A548B55884E894F8C508D51FD
:100BED008154885489558A4E8B4F8C508D51306964
:100BFD0020C3E53394034019E542A2E713F8E55508
:100C0D00F4240138400B20E7087554FFF42401F556
:100C1D00558154E8FAD3E813FC8852C3EF9403606E
:100C2D0020EF20E007E82CF8ECFA8140E8282402B8
:100C3D00F87AFEC3EF940340088A54884E8C508195
:100C4D005488548A4E8C50E56BC3335002646BF557
:100C5D006B306002815E753402D26043E680E52D13
:0F0C6D0054066026A840A941C3E913F9E813F81B
:100C7C00C2AF53E67F759100C3E498F594E499F5FF
:100C8C0095759104D26043E680D2AF22D26575444B
:100C9C0000752000306B03752040020CB7D26575CF
:100CAC004400752040306B03752000D2AF780120D2
:100CBC006722E52D54066002C265C3E541940540E8
:100CCC0013780294054008780394054002780630A6
:100CDC006902780A206019E544601530690AC3E599
:100CEC003394034003D53406D2AFD26CA1889166FD
:100CFC00D2AF0000C2AF206726E541C3FB940F4082
:100D0C00027B0FEB240530730123306A0274282018
:100D1C00620123F93069027982E58BC39940B505EC
:100D2C0044E59B5440B52002A17230690A08C3E81F
:100D3C00940A40010881E020650281B7C26553E640
:100D4C007F7591003067107594007595FE75910450
:100D5C00D26043E68081B7AE40AF41C3E49EF594C8
:100D6C00E49FF595A159C3E5339402500281B73045
:100D7C00650281B7D802A18681E0C26C53E67F750B
:100D8C009100855494855595759104854E56854FE3
:100D9C0057D26043E680D2AFE52D54066008206A36
:100DAC00020533020DC2306C0D206B0A206507154D
:100DBC0081158102161222780030640530650278A4
:100DCC0001E53775F007A4F9E5F028F5F0E9A2F094
:100DDC0013A2F113A2F213F537C3947850037537AD
:100DEC0078C3E53795384008D266C295C294C29351
:100DFC00306002A1FC855056855157D26043E68085
:100E0C0022207D11C2AF754302D291C292D2AF752E
:100E1C009F11020FDCC2AF754302D291C290D2AFC8
:100E2C00759F11020FDC307243207D20C2AF7543D9
:100E3C000390013E757E02C293D290306204D2942C
:100E4C00C150C291D2AF759F01020FDCC2AF754386
:100E5C000390013E757E02C295D292306204D29408
:100E6C00C170C291D2AF759F21020FDC207D17C2D9
:100E7C00AF754303900119C293306202D294D2AF82
:100E8C00759F01020FDCC2AF754303900119C29527
:100E9C00306202D294D2AF759F21020FDC207D11FB
:100EAC00C2AF754304D292C290D2AF759F21020F8C
:100EBC00DCC2AF754304D290C292D2AF759F0102CF
:100ECC000FDC307243207D20C2AF75430590012D9D
:100EDC00757E04C294D291306204D295C1ECC29258
:100EEC00D2AF759F11020FDCC2AF75430590014F55
:100EFC00757E01C294D291306204D293E10CC290FF
:100F0C00D2AF759F11020FDC207D17C2AF75430560
:100F1C0090010FC294306202D295D2AF759F11022C
:100F2C000FDCC2AF754305900123C2943062EBD243
:100F3C0093D2AF759F11020FDC207D11C2AF7543A8
:100F4C0006D290C291D2AF759F01020FDCC2AF7571
:100F5C004306D292C291D2AF759F21020FDC307240
:100F6C0042207D20C2AF75430190014F757E01C2B6
:100F7C0095D292306204D293E188C290D2AF759F21
:100F8C0021020FDCC2AF75430190012D757E04C2A6
:100F9C0093D290306204D295E1A8C292D2AF759FE1
:100FAC0001E1DC207D16C2AF754301900123C2958F
:100FBC00306202D293D2AF759F21E1DCC2AF754390
:100FCC000190010FC293306202D295D2AF759F018E
:100FDC00C2662290010D757E00C295C294C293D256
:100FEC0092D291D290C26222788076070876070856
:100FFC0076010876040876FF0876FF08760A0876EC
:10100C0002087601087601788C760108760008765D
:10101C00B40876FF0876FF0876FF0876030876FF9B
:10102C000876010876FF0876250876D008767808C9
:10103C0076C80876040876FF0876010876000876EC
:10104C007A08760A0876010876010876000876FF99
:10105C00227887E6FFC2727888C27DE630E102D240
:0F106C007DC27E7889E630E102D27EC3EF940226
:10107B006008758E01D27302108A758E00C27322BE
:10108B007880E6149000809378A4F67881E614902B
:10109B0000809378A5F67886E61490008D9378A659
:1010AB00F6789FE6F8700108C3E8941140027811B6
:1010BB00E82828F56E256E256E28F56F256E2828F5
:1010CB00F570789CE67538FF75390CB402067538E7
:1010DB00A075390AB4030675388275390578A3E60D
:1010EB001490009A93F569120FDF22227896E6FA94
:1010FB007897E6FB7888E6B40305C3EB940EFB30D8
:10110B007F047A007BFFC3EB9AFCC3948250027C72
:10111B00827575000575EC8575F0A4C3E5F0947DBB
:10112B0040F222D27F11F71205637A007B007C100C
:10113B00120559E55F2AFA74003BFBDCF37C04C310
:10114B00EB13FBEA13FADCF7FEC27F11F722E5EF94
:10115B0020E6037520000520903FFFE52014600674
:10116B00901DFF1460009304600375EF1253D9BFF9
:10117B007581C043FF8012055475EF0243B203E53E
:10118B00B3240420E70DF521E5E320E0068521B328
:10119B0043E301120FDF7580FF75A40075F19075A5
:1011AB00D47F75908775A5BF75F2BF75D50075A6F1
:1011BB000175E241E4F8F6D8FD756B01120FF412DC
:1011CB00165A78988676753001C2AF12056D1205E6
:1011DB007D12056312058412056312058B120563DC
:1011EB0012177D12056D12056D120568C2AF78FAE4
:1011FB0079FA308707D9FBD8F7021C00115D118BE8
:10120B0011F611F778988676120FDF75885075896D
:10121B001275C82475910475D84075A82275B8024B
:10122B0075E690759B80759D0075D10E75BC5875D4
:10123B00BB0675BA1175E880120554D2AF1208AC13
:10124B0053DACF207E0343DA20307E0343DA104398
:10125B00DA01C2D8C27112056DD2617B037A0CE53B
:10126B005E70077A0CDB030211F712056320700323
:10127B000211F7C270E55FC3940240E1E52F541FE2
:10128B00856160F561B560D5DAD5C26153DACF20DF
:10129B007E0343DA20307E0343DA10C2D8C2717862
:1012AB00A2E67008D274E52F54E0F52FC2757529AC
:1012BB0000120568307409C3E529940A4002D275FF
:1012CB0012055978023074027800C3E55F9840F03C
:1012DB00C2AF12057D12057D12057DD2AF12056DD1
:1012EB00754D00120559788CE6C394015003021317
:1012FB00C4E530C3940150030213C4207435C3E515
:10130B005F94FF50030213C4C2AF120592D2AF1207
:10131B000568C3E55F940150EFC2AF12057D12055E
:10132B005E12057DD2AF120568C3E55F94FF40E9FD
:10133B000218027F05D27F11F7120568C2AFC27F78
:10134B0011F7AE5FC3E55F947FD2AF4076120554C1
:10135B00C2AF120592D2AFDFDC312EC3EE9405780B
:10136B0097F612056D12169C1217857F0AD27F1104
:10137B00F7120568C2AFC27F11F7AE5FC3E55F948A
:10138B007FD2AF50E6120554C2AF12057D12055E37
:10139B0012057DD2AFDFD6312EEE24057896F612EC
:1013AB00056D12169C1217B412056811F7C3E55F91
:1013BB0094FF50026106021802C3E55F954D40038E
:1013CB00855F4D12056878017988E7B403027805CB
:1013DB00C3E55F98400241EEC2AF1205921205922F
:1013EB00120592D2AF12056D753000E4F531F5326E
:1013FB000531E531F470390532789AE678191460C5
:10140B0012783214600D787D14600878FA1460033A
:10141B00753200C3E53298401715327531B478999F
:10142B008676C2AF120592D2AF789886761205688F
:10143B0012055EE52A700530740221F778012074DD
:10144B00027806C3E55F9840A7120568E52A70038A
:10145B000211F7C2AF120FDFE4F522F523F524F5E5
:0F146B0025F526F56AD2AF7885E6C333F568E438
:10147A00F545F546F547F548F549F573F52CF52D8B
:10148A00F53775730875BB1012055412093FE5E864
:10149A0020ECFBA8BDA9BEE97001F88874120943C3
:1014AA0075730875BB107887E6FE7602115D78873A
:1014BA00EEF6C2AF7564FF1209FE852264852265C5
:1014CA00852266D2AF75220175240175250175261C
:1014DA000185636C756D017888E6B40307C27D30B7
:1014EA007602D27DD268D269753300120F45120F87
:1014FA006A120A1E120A25120A1E120A25120A1E48
:10150A00021519C2AF115DD2AF75730075BB061211
:10151A000CA912065D120DC3120E0D120A25120C29
:10152A0098306D031206FD20670312084F306703D7
:10153A00120896120DC3120E32120A25120CA93085
:10154A006D03120739120DC3120EA9120A25120CC5
:10155A0098306D03120797120DC3120ECE120A2588
:10156A00120CA9306D031207F4120DC3120F4512A3
:10157A000A2512093F120C98120DC3120F6A12099A
:10158A0043120A2530692F206B2C856764856765AD
:10159A0085636C756D0179187A0CC3E53399400936
:1015AA00C269D26A8A350215C0C3E55F9401400355
:1015BA0002151902161A306A1B206B18E5351470C9
:1015CA0004C26AA10DF535C3E55F94014003021513
:1015DA001902161A753600C3E56294014009856737
:1015EA006585636C756D01C3E56278FA98502130A0
:1015FA007404E52A601A78F0306B058567647820F0
:10160A00C3E541985002A1190536E55F6002C11D84
:10161A00753600C2AF120FDF7887E6FE7602115DDB
:10162A007887EEF6E4F522F523F524F525F526F577
:10163A0068C268D2AF120554120FDF307406E52A69
:10164A00700221F7788DE6C39401400241CB61F61E
:10165A00901A0D78201216DEE520B4A50CA31216F6
:10166A00DEE520B45A0302167C120FF412169C020D
:10167A00169B901A0378807B0A1216DEA308DBF900
:10168A00901A0F788C7B181216DEA308DBF9901AD1
:10169A002722C2AF12171D1216F7901A00740E12E3
:1016AA0016E3A374041216E3A374141216E3901A31
:1016BA000378807B0A1216E2A308DBF9901A0F78E6
:1016CA008C7B181216E2A308DBF912173012170ED8
:1016DA00901A2722E493F622E6438F01538FFD7571
:1016EA00EF0275B7A575B7F1F0538FFE22438F024B
:1016FA00438F0175EF0275B7A575B7F1901A0DF012
:10170A00538FFC22901A0D74A5D1E3901A0E745AC5
:10171A00D1E3227A3079D07820901A40D1DEE520C0
:10172A00F709A3DAF7227A3079D0901A40E7D1E3A1
:10173A0009A3DAF922AB77A878BB01027980BB0248
:10174A00027981BB03027982BB04027994BB050248
:10175A007983BB06027986BB07027992BB080279B4
:10176A0087BB0902799CBB0A027988BB0B0279897B
:10177A00E8F7227C0512056DDCFB22C2AF12057D5B
:10178A0012058412058B12059212055E12057D124E
:10179A00058412058B12059212055E12057D12054B
:1017AA008412058B120592D2AF22C2AF1205921291
:1017BA00058B12058412057D12055E12059212052B
:1017CA008B12058412057D12055E12059212058B95
:1017DA0012058412057DD2AF22AE77AF78C2AF125E
:1017EA00057D12057D12057D12055EDEF212059257
:1017FA0012055EDFF8D2AF2212178512177D121773
:10180A007D7577017578017579001217E37C05AD4E
:10181A005F12056DC3ED955F70F5C3E55F940140F6
:10182A000AC3E55F94FF403702184612173F1216A3
:10183A009C121785C2AF75EF1212177DDCD105799C
:10184A00C3E5799403500280C112177D0578E577C4
:10185A001490009F93F808C3E57898500280A81264
:0E186A00177D12177D0577C3E577940C5002A9
:101878008094120FF412169CC2AF75EF1212177DE6
:0319FD000211597B
:101A00000E041407070104FFFF0A020101A55A0191
:101A100000B4FFFFFF03FF01FF25D078C804FF01DA
:081A200000FF0A010100FFFFB5
:101A400023585031384123202020202020202020DE
:101A500023424C48454C4923463333302320202031
:101A60002020202020202020202020202020202076
:101C0000C2AFC2D353D9BF7581C043B20343FF8073
:101C1000752438752503B1C975EF0275E24043F1AB
:101C20008053A47F75D400D2877DFA780379E67C4F
:101C300010752200752300901DD67B0675249875BB
:101C400025013087028142208708D8FBD9F9DCF7CB
:101C500081B4308708D8FBD9F9DCF781B4B189E4C5
:101C600093A3C39A6004DDC381B4DBDBB17B600264
:101C7000812B7B08E493FAA3B15CDBF87A30B15C8A
:101C8000752200752300B17BEAFCEBFDC3ED94FEE9
:101C9000400EB17B8A278B28ED30E0048A828B834B
:101CA000B17B7AC270D8C3ED94FE601350CEBD00F4
:101CB00025EC60097520007521FF0200008100A855
:101CC00027A9280809D804D90281D3B17FEA89AAB3
:101CD000F281C50D81A0C3ED94035049EDA2E092BD
:101CE000007AC5C3E5829400E583941C50902000DF
:101CF00010438F02438F0175B7A575B7F1F030001F
:101D00001FA827A9280809438F01538FFDD804D99C
:101D100002A12089AAE275B7A575B7F1F0A3A10DBC
:101D2000538FFC817C7AC1BD030CE493A3FAB140CC
:101D3000DCF8B138817C817EAA22AB23B15CEBFA5E
:101D4000EA6222752608C3E52313F523E52213F57D
:101D50002250066323A0632201D526EAB1C9B1C986
:101D600075260AEAF4200102D287300102C287B147
:101D7000C9C3134002C201D526EB22B17FEAFB2082
:101D80008702A17F308702A184752608AE24AF2583
:101D9000C3EF13FFEE13FEB1CDB1C9C3EA13308711
:101DA000024480FA30E703632201C3E52313F523DD
:101DB000E52213F52250066323A0632201D526D91C
:101DC000E52265236523F52222AE24AF250E0FDE22
:101DD000FEDFFCD20122424C48656C693437316326
:041DE000F3300601D5
:00000001FF
